:04040000020485323B
:01040B0032BE
:0104130032B6
:01041B0032AE
:0104230032A6
:01042B00329E
:010433003296
:01043B00328E
:010443003286
:01044B00327E
:010453003276
:01045B00326E
:03046300020DDDAA
:01046B00325E
:010473003256
:03047B000205AEC9
:0A04DE007800E4F208F208F208F2D8
:0305120002047E62
:05047E001205E080FE04
:0E05150012149D120E02AA82AB83ACF0FD7888
:0A05230000D3E29AF4B3F508B30820
:0C052D00E29BF4B3F509B308E29CF4B3C0
:0A053900F50AB308E29DF4F50B90FB
:0E0543001539E493FE740193FF740293FA7469
:0C0551000393FB78047402F208E4F20843
:0E055D00F208F28E828F838AF0EB120904AA54
:0B056B0082AB83ACF0FDC3E5089AE50D
:06057600099BE50A9CE56B
:0C057C000B9D402DE5FF035401FAB40173
:010588000072
:0A058900E433FA600543FF0280032B
:0305930053FFFD16
:0C059600120E02AA82AB83ACF0FD7800CC
:0B05A200EAF208EBF208ECF208EDF2C0
:0105AD00222B
:0E05AE00C0E0C002C0D075D000E58A30E21D6A
:0A05BC00E5FF03035401FAB4010047
:0A05C600E433FA600543FF048003EC
:0305D00053FFFBDB
:0605D300538AFB53E8F718
:0705D900D0D0D002D0E032C7
:0E05E000438D04438C02758A00439A1075E81F
:0B05EE0000120A74120E69C2F085F0C2
:0805F900221208EED2F085F099
:0A0601002275820C1206F743A88050
:07060B00120A80120515120E
:040612000C8980F5DA
:04153900F4010000B9
:07061600AA827418B502006E
:03061D0050012267
:0D062000EA240983C0E0EA241C83C0E02224
:02062D005F6705
:02062F006F77E3
:020631007F87C1
:02063300F6F6D9
:02063500F6F6D7
:020637008F979B
:020639009FA779
:02063B00AFB757
:02063D00BFC735
:02063F00F6F6CD
:02064100CFD711
:02064300DFE7EF
:01064500EFC5
:020646000606A6
:020648000606A4
:02064A000606A2
:02064C000606A0
:02064E0006069E
:0206500006069C
:0206520006069A
:02065400060698
:02065600060696
:02065800060694
:02065A00060692
:02065C00060690
:01065E000695
:08065F00A210928043FD01226C
:08066700A210928143FD022262
:08066F00A210928243FD042257
:08067700A210928343FD08224A
:08067F00A210928443FD102239
:08068700A210928543FD202220
:08068F00A210929043FE01222B
:08069700A210929143FE022221
:08069F00A210929243FE042216
:0806A700A210929343FE082209
:0806AF00A210929443FE1022F8
:0806B700A210929543FE2022DF
:0806BF00A210929643FE4022B6
:0806C700A210929743FE80226D
:0806CF00A21092A043FF0122DA
:0806D700A21092A143FF0222D0
:0806DF00A21092A243FF0422C5
:0806E700A21092A343FF0822B8
:0706EF00A21092A443FF10CA
:0106F60022E1
:0706F700AA827418B502008D
:0306FE0050012286
:0D070100EA240983C0E0EA241C83C0E02242
:02070E00404F5A
:020710005E6D1C
:020712007C8BDE
:020714005C5C2B
:020716005C5C29
:020718009AA99C
:02071A00B8C75E
:02071C00D6E520
:02071E00F403E2
:020720005C5C1F
:020722001221A2
:02072400303F64
:010726004E84
:020727000707C2
:020729000707C0
:02072B000707BE
:02072D000808BA
:02072F000808B8
:020731000707B8
:020733000707B6
:020735000707B4
:020737000708B1
:020739000808AE
:02073B000808AC
:02073D000808AA
:01073F0008B1
:08074000301005538FFE800309
:03074800438F01DB
:04074B0053FDFE223A
:08074F00301005538FFD8003FB
:03075700438F02CB
:04075A0053FDFD222C
:08075E00301005538FFB8003EE
:03076600438F04BA
:0407690053FDFB221F
:08076D00301005538FF78003E3
:03077500438F08A7
:0407780053FDF72214
:08077C00301005538FEF8003DC
:03078400438F1090
:0407870053FDEF220D
:08078B00301005538FDF8003DD
:03079300438F2071
:0407960053FDDF220E
:08079A0030100553F6FE800348
:0307A20043F6011A
:0407A50053FEFE22DF
:0807A90030100553F6FD80033A
:0307B10043F6020A
:0407B40053FEFD22D1
:0807B80030100553F6FB80032D
:0307C00043F604F9
:0407C30053FEFB22C4
:0807C70030100553F6F7800322
:0307CF0043F608E6
:0407D20053FEF722B9
:0807D60030100553F6EF80031B
:0307DE0043F610CF
:0407E10053FEEF22B2
:0807E50030100553F6DF80031C
:0307ED0043F620B0
:0407F00053FEDF22B3
:0807F40030100553F6BF80032D
:0307FC0043F64081
:0407FF0053FEBF22C4
:0808030030100553F67F80035D
:03080B0043F68031
:04080E0053FE7F22F4
:0808120030100553F7FE8003CE
:03081A0043F701A0
:04081D0053FFFE2265
:0808210030100553F7FD8003C0
:0308290043F70290
:04082C0053FFFD2257
:0808300030100553F7FB8003B3
:0308380043F7047F
:04083B0053FFFB224A
:08083F0030100553F7F78003A8
:0308470043F7086C
:04084A0053FFF7223F
:08084E0030100553F7EF8003A1
:0308560043F71055
:0308590053FFEF5B
:01085C002279
:07085D00AA827418B5020025
:0508640050030208E151
:0D086900EA240983C0E0EA241C83C0E022D9
:02087600A8AB2D
:02087800AEB11F
:02087A00B4B711
:02087C00E1E1B8
:02087E00E1E1B6
:02088000BABDFF
:02088200C0C3F1
:02088400C6C9E3
:02088600CCCFD5
:02088800E1E1AC
:02088A00D2D5C5
:02088C00D8DBB7
:01088E00DE8B
:02088F00080857
:02089100080855
:02089300080853
:02089500080851
:0208970008084F
:0208990008084D
:02089B0008084B
:02089D00080849
:02089F00080847
:0208A100080845
:0208A300080843
:0208A500080841
:0108A7000848
:0308A800A2802209
:0308AB00A2812205
:0308AE00A2822201
:0308B100A28322FD
:0308B400A28422F9
:0308B700A28522F5
:0308BA00A29022E7
:0308BD00A29122E3
:0308C000A29222DF
:0308C300A29322DB
:0308C600A29422D7
:0308C900A29522D3
:0308CC00A29622CF
:0308CF00A29722CB
:0308D200A2A022BF
:0308D500A2A122BB
:0308D800A2A222B7
:0308DB00A2A322B3
:0308DE00A2A422AF
:0208E100C32230
:0708E30030100453F7DF227F
:0408EA0043F720228E
:0708EE0030100453F7BF2294
:0408F50043F7402263
:0708F90030100453F77F22C9
:0409000043F7802217
:0E090400AA82AB83ACF0FD33E433FE6013C374
:0A091200E49AF50CE49BF50DE49C5B
:08091C00F50EE49DF50F8008C3
:050924008A0C8B0D8C14
:030929000E8D0F21
:05092C00AA0CAB0DACAC
:040931000EAD0F7880
:0A09350007E233E433FF602078048A
:0C093F00E2D3F43400F50C08E2F43400BC
:0A094B00F50D08E2F43400F50E0883
:08095500E2F43400F50F8011FB
:08095D007804E2F50C08E2F554
:080965000D08E2F50E08E2F5B1
:01096D000F7A
:07096E00780CE50CF208E52E
:080975000DF208E50EF208E5A1
:0C097D000FF28A828B838CF0EDC006C064
:0C098900071209D87808C0E0E582F208E7
:0E099500E583F208E5F0F2D0E008F2D007D0DA
:0C09A30006EF6E60207808E2D3F4340008
:0E09AF00FE08E2F43400FF08E2F43400FA0817
:0B09BD00E2F434008E828F838AF02267
:0C09C8007808E2F58208E2F58308E2F509
:0409D400F008E22223
:0C09D800AA82AB83ACF0FD7810EAF208B4
:0E09E400EBF208ECF208EDF27E007F007A00E4
:0409F2007B007C20EA
:0709F6007813E23392007850
:0C09FD0010E225E0F208E233F208E233D9
:0E0A0900F208E233F2EE2EFEEF33FFEA33FA8C
:090A1700EB33FB30000343060140
:0C0A2000780CC3E2F5F0EE95F008E2F56A
:0E0A2C00F0EF95F008E2F5F0EA95F008E2F53B
:0C0A3A00F0EB95F04022780CD3E29EF423
:0E0A4600B3FEB308E29FF4B3FFB308E29AF4E4
:0C0A5400B3FAB308E29BF4FB7810E24414
:020A600001F2A1
:0C0A6200DC927810E2F58208E2F58308CF
:060A6E00E2F5F008E222AF
:0604B400E478FFF6D8FD1C
:080492007909E94400601B7ABE
:05049A00019015D1786E
:03049F005D7593F5
:0A04A200F0E493F2A308B80002058D
:0804AC0093D9F4DAF27593FF15
:0504E80078147480F29D
:070A7400120A95120A831219
:050A7B000E23020E62D3
:030A8000020B174F
:030A830053BEFB64
:0E0A8600E5BE30E6FB75C68043BE0475C700B2
:010A9400223F
:0A0A950075FF0075A00675F79922A1
:0C0A9F00120E02AA82AB83ACF0FD7814AA
:0A0AAB00D3E29AF4FA7419B50200C0
:0C0AB5005038E5FFA2E49202400943FF24
:070AC10010758202121531CD
:0E0AC80053F7EF53FFEF758201121531A2A410
:0A0AD600920143F71030020343FFC2
:010AE0001005
:0C0AE100120E02AA82AB83ACF0FD781468
:020AED00EAF22B
:010AEF0022E4
:0E0AF000C2AF75D69F75820A12153175FF00D0
:0E0AFE0075FE0075FD0075F50075F40075F3CA
:0B0B0C0000900064120E2E0200062272
:0E0B1700E5FF20E20C75820A12153130A203B0
:030B2500020AF0D1
:010B280022AA
:060B2900120A9FA2012246
:030B2F00A2A3225C
:040B320053FFFE224D
:060B3600D2A043FF0122E2
:0604ED00751000C203C2FD
:0604F300047815E4F27824
:0904F90016E4F2781774FFF27AA0
:04050200C17B0B7836
:0605060018EAF208EBF216
:0C0B3C00782C740AF275820112143978CA
:0B0B48002D7440F275820412146B78CB
:0B0B53002C7440F275820412143978F3
:050B5E001774FFF222F4
:0E0B630090F051E0FA53027FBA215190F05504
:0E0B7100E0FAA3E0FB4A6006BA0143BB004075
:0A0B7F0090F052E0FABA2002800A5A
:050B8900BA21028014F6
:050B8E00BA222E801EBA
:070B9300782A745DF208747A
:080B9A00F0F2900007021404C0
:070BA2007828745DF208746D
:080BA900F0F29000070213E3D3
:0C0BB10090F053E0FAA3E07815EAF2029D
:020BBD001425FD
:010BBF002213
:010BC0002212
:010BC1002211
:0C0BC2007818E2F58208E2F58312048343
:0E0BCE0090F05DE0FAA3E0FBA3E0FCA3E0FDE5
:0D0BDC00BA4D1DBB011ABC0017BD0014204E
:050BE9000411D204120A
:0E0BEE000E02AA82AB83ACF0FD90F030EAF06C
:010BFC0022D6
:0A0BFD0090F064E0FABA10028004E0
:040C070075820022D0
:0E0C0B0090DE0E7404F090DE14E0FA30E00784
:070C190090DE16E0F58222D7
:040C200075820022B7
:0E0C240090DE0E7404F090DE28E0FA90DE16EA
:0C0C3200E0FB700890DE14E0FB54FEF0C4
:050C3E00D2068A8222AB
:0A0C4300AA82AB83781A7922E2F34B
:0B0C4D007823EAF208EBF27582041233
:0E0C58000E6A90DE16E0FA700890DE14E0FAE4
:030C660054FEF049
:010C69002268
:0E0C6A0090DE0E7404F090DE11E0FA4401F00A
:080C78007440B51003D38001A4
:010C8000C3B0
:060C81009203751000D281
:020C8700062243
:070C8900120EE230041B1201
:0E0C90000E02AA82ACF0FD90F030E0FBEAC349
:070C9E009BFA7446B5020049
:050CA5005003120AF0EB
:0A0CAA0090F064E0FABA1002800135
:010CB400221D
:0B0CB50090DE0E7404F0E510700B30B0
:0A0CC000030B90DE11E0FA20E103BF
:030CCA00120C6A9F
:0A0CCD0090DE0E7401F0781679171E
:080CD700E2F5F0E3B5F00122A3
:0E0CDF0090DE11E0FA20E03A90DE2274A1F0DF
:0E0CED007420F0E4F0E4F090DE22F0E4F07405
:0C0CFB0002F0E4F0781690DE22E2F090A7
:0C0D0700DE22E4F090DE11E04401F07800
:0A0D130016E25483F27816E2FA7833
:040D1D0017F2D206F1
:010D210022AF
:0A0D220090F064E0FABA10028004B9
:040D2C0075820022AA
:0E0D300090DE0E7404F090DE11E0FA30E11057
:080D3E00EA30E0047582002296
:080D46007440C39510F58222F0
:080D4E007480C39510F58222A8
:040D5600AA82AB833F
:0A0D5A00781BE260527440C395104C
:070D6400FC781BE2B504005E
:060D6B005004781BE2FCBD
:0A0D71007825ECF27826EAF208EB90
:0E0D7B00F2758204C002C003C004120E9FD0A5
:0C0D890004D003D002EC2AFAE43BFB7813
:090D95001BE2C39CF2EC2510F5F1
:0A0D9E00107440B510B6C002C00387
:090DA800120C6AD003D00280A9EC
:010DB100221F
:0B0DB200E58290DE28F005107440B5CB
:050DBD001003020C6AA6
:010DC200220E
:060DC3007815E2F5822222
:0A0DC900AA827816E2547C4A7816DC
:020DD300F2220A
:080DD500AA827816E24AF2221C
:0E153D001201000202000020FB1F002200002D
:04154B000102030195
:0E154F0009024300020100C03209040000013D
:0E155D00020201000524002001042402020500
:0E156B00240600010524010001070581030A82
:0E157900000109040100020A00000007050439
:0B158700024000000705840240000045
:011592000454
:041593000403090440
:0E159700260350006F006C006F006C007500A2
:0E15A500200043006F00720070006F007200A3
:0A15B3006100740069006F006E0013
:0C15BD000C0357006900780065006C000A
:0215C900931578
:0215CB00971572
:0215CD00BD154A
:0215CF00E60331
:0715D1008025000000000866
:0804BA007830E84400600A7983
:0304C2000075932F
:0604C500F0E4F309D8FC8D
:0804CB00782DE84400600C7973
:0B04D3000190F000E4F0A3D8FCD9FA7F
:0C0DDD00C0E0C000C0D075D000781CE25F
:0E0DE9002401F208E23400F208E23400F208BD
:0B0DF700E23400F2D0D0D000D0E03297
:0C0E0200A2BCE433FAC2BC781CE2FB087E
:0E0E0E00E2FC08E2FD08E2FEEA24FF92BC8B43
:070E1C00828C838DF0EE22B1
:0B0E230075EDBBD2BC75EBFAD2AF221C
:040E2E00AA82AB8366
:090E32008A048B051ABAFF011BAA
:0E0E3B00EC4D60227582FAC002C00312153120
:0E0E49007582FA1215317582FA121531758212
:0A0E5700F9121531D003D00280D14A
:010E6100226E
:070E620075D23175D3F022B7
:04050C00C205C2065C
:010E69002266
:0E0E6A00AA82E4CA25E0CA33FB74202AFA7477
:0A0E7800DE3BFB7822E2FC7823E267
:040E8200FD08E2FE87
:0E0E8600EC60131C8A828B83E0FF8D828E83CA
:080E9400F0A3AD82AE8380EAF9
:030E9C00D2062259
:0E0E9F00AA82E4CA25E0CA33FB74202AFA7442
:0A0EAD00DE3BFB7825E2FC7826E22C
:040EB700FD08E2FE52
:0E0EBB00EC60141C8D828E83E0FFA3AD82AE2E
:090EC900838A828B83EFF080E93B
:010ED20022FD
:0C0ED300C20590DE017401F090DE0B748B
:030EDF0007F022F7
:0C0EE200120B29400E53BE7F120B329001
:070EEE00F064E4F0C20522EC
:0E0EF50090F064E0FA7013120B3643BE8000DA
:0C0F030000000090F0647402F0120ED3A5
:0E0F0F0090DE06E0FA90DE02E0FBEA30E0023F
:020F1D00D205FB
:0E0F1F00EA30E21690F0647404F090F065E49D
:0C0F2D00F0C002C003120ED3D003D002AB
:060F3900EA30E102C205EE
:050F3F00EB20E001229F
:0C0F440090DE0EE4F090DE11E0FAD20620
:0E0F5000EA30E40B90DE117480F090F065E45E
:010F5E00F0A2
:0D0F5F00EA30E20990DE11E4F090F065F058
:070F6C00EA20E003021095EA
:0A0F730090F065E0FBBB0102800373
:030F7D0002101B44
:0E0F800090DE16E0FB90F059E0FCA3E0FD8B44
:0C0F8E00067F00C3EC9EED9F50028C0318
:070F9A007822EBF2782079C8
:0C0FA10023E2F308E209F3758200C002AD
:0C0FAD00C003120E6AD003D0027820E2CC
:0E0FB9002BF208E23400F27C0090F059E0FDCB
:0E0FC700A3E0FE90F059EDC39BF0EE9CA3F06A
:0E0FD50090F059E0FBA3E0FC4B600990DE11A8
:060FE3007440F0021095BD
:0E0FE90090F051E054606007C002120BC2D0BD
:010FF70002F7
:0D0FF80090DE0EE4F090F065E0FB700990D3
:08100500DE117468F002109581
:0E100D0090DE117448F090F065E4F00210954A
:0C101B0090DE16E0FBBB086C7822740825
:08102700F278237451F2087401
:0C102F00F0F2758200C002120E6AD002BE
:0E103B0090F065E4F090F051E054607009C050
:0810490002121100D002800721
:07105100C002120B63D00284
:0D10580090DE0EE4F090F065E0FB70089073
:07106500DE117460F0802928
:0E106C00BB012690F059E0FBA3E0FC4B6008AE
:08107A0090DE117440F08013B8
:0D10820090DE11744AF090F065E4F08006F5
:06108F0090DE117440F038
:0D109500EA20E16690F065E0FBBB025E9092
:0E10A200F059E0FBA3E0FCC3EB9420EC9400BB
:0B10B00050097A0A90F065E4F080041B
:0410BB007A027B201A
:0710BF007825EBF27820799F
:0C10C60026E2F308E209F3758200C00284
:0E10D200C003120E9FD003D00290DE11EAF090
:0C10E0007820E22BF208E23400F27A00E3
:0E10EC0090F059E0FCA3E0FD90F059ECC39B9E
:0510FA00F0ED9AA3F0E7
:0110FF0022CE
:0A11000090F05BE4F090F05CF090DA
:09110A00F052E0FA740CB5020089
:0311130050012266
:07111600EA2A2A90111D7363
:07111D000212C902137E0259
:06112400139002137E028D
:06112A00139002121302F3
:06113000114402139002BD
:06113600126C02123102EE
:06113C00128E0213900266
:02114200138117
:0E11440090F053E0FAA3E0FBFC7D00BC010537
:05115200BD0002801346
:08115700BC0205BD000280206E
:08115F00BC0305BD000280394C
:031167000211E290
:07116A007820743DF20874C7
:0C11710015F290F0597412F0A3E4F002A3
:02117D0011ED72
:04117F00EA600122FF
:071183007820744FF208749C
:0C118A0015F2901551E493FCA3E493FDD2
:0A11960090F059ECF0A3EDF0804D4D
:0E11A0008A047D00901592E493FE7F00C3EC5C
:0611AE009EED9F400122AE
:0C11B400E4CA25E0CA33FBEA24C9F58236
:0C11C000EB3415F583E493FAA3E493FBF1
:0C11CC007820EAF208EBF28A828B83E0C4
:0A11D800FA90F059F0A3E4F0800B48
:0B11E200120BC090F065E0FA700122D3
:0E11ED0090F057E0FAA3E0FB90F059E0FCA36D
:0E11FB00E0FDC3EA9CEB9D500890F059EAF02D
:03120900A3EBF064
:07120C0090F0657402F0226E
:0E12130090F053E0FAA3E0FB90DE00EAF0EA70
:0612210060047A0880025F
:021227007A0447
:0812290090F064EAF0021425C4
:0E12310090F053E0FAA3E0FBBA0005BB000208
:02123F00800825
:08124100BA0124BB0021801456
:0A12490090F064E0FA7408B50200AA
:0A125300501490F0647408F0800C51
:0B125D0090F0647410F0120B3C800154
:011268002263
:0312690002142547
:0C126C0090F064E0FABA10047A018002ED
:021278007A00FA
:08127A0090F05BEAF0782874A3
:0A1282005BF20874F0F29000010224
:02128C0013E36A
:08128E0090F064E0FABA1000D0
:03129600500122E2
:0B12990090F055E0FAA3E0FB7C4F7DD5
:0C12A400158C828D83A3A3A3A3E493FC0C
:0A12B0007D00C3EA9CEB9D40012283
:0712BA007828745BF2087450
:0812C100F0F29000010213E3BA
:0E12C90090F051E0541FFA7B00BA0005BB0004
:0312D7000280147E
:0812DA00BA0105BB0002802BE4
:0912E200BA0206BB00030213531B
:0312EB0002137D6E
:0912EE00120B2F50047A0180025A
:0212F7007A007B
:0812F90090F05BEAF078287424
:0A1301005BF20874F0F290000202A3
:02130B0013E3EA
:08130D0090F064E0FABA100050
:0E131500500C90F055E0FAA3E0FB4A60012274
:0B13230090F055E0FAA3E0FB7C4F7D4A
:0C132E00158C828D83A3A3A3A3E493FC81
:0A133A007D00C3EA9CEB9D400122F8
:071344007828745BF20874C5
:08134B00F0F29000020213E32E
:0E13530090F053E0FAA3E0FBEA540F60028032
:01136100018A
:011362002268
:0813630090F064E0FABA1000FA
:03136B005001220C
:07136E007828745BF208749B
:08137500F0F29000020213E304
:01137D00224D
:03137E0002142531
:071381007828745BF2087488
:08138800F0F29000021213E3E1
:01139000223A
:03139100A2052290
:0C139400AA8CA2BD9207C2BD438C10536E
:0213A0008CFEC1
:0E13A200758900C2C5D2BDABBE74FC5B4401B0
:0E13B000F5BE000000E5BE54036007D2904376
:0413BE008701C29051
:0913C200C2BDE58930E702C20555
:0C13CB00300509C002120B2FD00250CBDD
:0C13D700E5BE30E6FB8A8CA20792BD2226
:0E13E300AA82AB8390F0657402F090F059EA94
:0C13F100F0A3EBF07828E2FA08E2FB78A9
:0713FD0020EAF208EBF222E6
:0E140400AA82AB8390F0657401F090F059EA73
:0C141200F0A3EBF0782AE2FA08E2FB7885
:07141E0020EAF208EBF222C4
:0E14250090F0657401F090F059E4F0A3F0220D
:0614330090F065E4F022D8
:0C143900E58290DE0EF0782CE2FA7B00D9
:0E14450074072AFAE43BFBC423CAC423541FD5
:0C1453006ACA541FCA6ACA30E40244E0AE
:0C145F0090DE10EAF090DE127401F02222
:0C146B00E58290DE0EF0782DE2FA7B00A6
:0E14770074072AFAE43BFBC423CAC423541FA3
:0C1485006ACA541FCA6ACA30E40244E07C
:0C14910090DE13EAF090DE157401F022EA
:0115D8000012
:0115D9000011
:02048300E47320
:02051000C2081F
:05149D0010060280159D
:0A14A20090DE0CE0FA782EF220082C
:0A14AC000AD20890DE0CE0FA782F57
:0114B600F243
:0C14B700121391400790F064E0FA7004FA
:0414C30053FFEF22C2
:0C14C700BA103D30083690DE0CE0FA7BD5
:0C14D30000782FE2FC7D00EAC39CFAEBDD
:0B14DF009DFBEA30E60543FF10800390
:0314EA0053FFEFBE
:0C14ED0090DE0CE0FA782ED3E29AF4FABC
:0514F9007460B5020063
:0514FE00501DC2082290
:0415030043FF102270
:0E150700120E02AB83ACF0FDEB035401FA6050
:051515000443FF102259
:03151A0053FFEF8D
:01151D0022AB
:030485007581225C
:0A04880012151EE582600302047ED7
:04151E0075820022B0
:0B1522000000000002152D000000007A
:04152D0000000000BA
:08153100E5826003D582EA2285
:00000001FF
